S123C000546869732070726F6772616D20697320636F707972696768742031393934202040
S123C02062793A2020202020202020202020202020204772616E742042656174746965200D
S123C040202045646D6F6E746F6E2C2020414220202020202043616E6164612020202020D1
S123C0602D2D2D2D2D2D2D2D2D2D2D2D2D2D2D2D416C6C2072696768747320202020202062
S123C0807265736572766564212020546869732070726F6772616D206D6179206E6F742033
S123C0A0626520636F70696564206F72202020207573656420696E2077686F6C65206F72B8
S123C0C0696E207061727420776974686F75742074686520657870726573736564202020C6
S123C0E07772697474656E20636F6E73656E74206F662074686520617574686F722E20209E
S123C1002A20202043414C4C45522D494420202A00313939372C204D2E2042656E6F697498
S123C12020002A20496E697469616C697A696E67202A002A202020204E6F6D732120202094
S123C14020202A002A20417474656E74652020202020202A002A206427617070656C2E2E25
S123C1602E2020202A0043686F6978204E6F6D3A2020202300212020426164202045505272
S123C1804F4D20202100212043616C6C20466163746F727920210012151515151512000417
S123C1A0080E111F100E008640B710398E00FFBDCDA98638B74000BDCDA98601B74000BD6E
S123C1C0CDA9860FB74000BDCDA98606B740008640BDCDA9B74000C608CEC197A60008BD54
S123C1E0CD8F5A26F7CEC19FC608A60008BDCD8F5A26F78601BDCDA9B74000BDCDAF1A83A7
S123C20077C42716CEC175BDCD9886C0BDCDA9B74000CEC186BDCD9820FECEC100BDCD9806
S123C22086C0BDCDA9B74000CEC111BDCD98CE00C8BDCD0B0926FA8601BDCDA9B74000CEF5
S123C240C122BDCD9886C0BDCDA9B74000CEC133BDCD98CEB610C60AA6008130240A8630E2
S123C260BDCD18BDCD2D200C813923088630BDCD18BDCD2D085A26E0C610A6008120240A8E
S123C2808620BDCD18BDCD2D200C817F23088620BDCD18BDCD2D085A26E0A60027074FBDFD
S123C2A0CD18BDCD2D088CB7DB25AB8606B7102B4FB7102C8604B7102D4F97049705970C81
S123C2C0970ECE000FDF08860197028600970D860197064FB710268640B710240EB6102E94
S123C2E0842026037EC67FB6102FD60DC11623037EC3AF58CEC2FC3AEE006E00C32AC34774
S123C300C389C3D2C409C438C45DC486C49AC4AFC4DEC506C57FC5A6C5DAC5F6C3AFC3AFD9
S123C320C3AFC3AFC61FC634C65681042609970A8601970D7EC67F818027037EC67F970A48
S123C3408607970D7EC67F8109260D97079B0A970A8602970D7EC36E811227078600970D7E
S123C3607EC67F97079B0A970A8603B7000D9604810A25127A0004CE000FC6BDA615A70029
S123C380085A26F8DF087EC67F813025228139221EDE08A70008DF089B0A970A7A000796A4
S123C3A007810127037EC67F8604970D7EC67F8600970DCE000F96042706C6153A4A26FCC3
S123C3C0DF087D000C2604C601D702960497057EC67F813025308139222CDE08A70008DFA4
S123C3E0089B0A970A7A00079607810A27037EC67F8605970DDE088603A70008860AA700D1
S123C40008DF087EC67F7EC3AF814F2707815027037EC3AFDE08C604E70008C601E7000838
S123C420A70008DF089B0A970A7A000727037EC3AF8606970D7EC67F8130251E8139221AA4
S123C440DE08A70008DF089B0A970A7A000727037EC67F8606970D7EC67F7EC3AF9B0A27F9
S123C460037EC3AF8600970D7D000C2604C601D70296044C97049705CE000FC6153A4A26C9
S123C480FCDF087EC67F810D24037EC3AF970B9B0A970A8608970D7EC67F810127037EC383
S123C4A0AF9B0A970A7A000B8609970D7EC67F810827037EC3AF97077A000B9B0A970A8676
S123C4C00A970D9604810A25127A0004CE000FC6BDA615A700085A26F8DF087EC67F813033
S123C4E025218139221DDE08A70008DF089B0A970A7A000B7A000727037EC67F860B970D0F
S123C5007EC67F7EC3AF8102271381042724810627358107273F810827507EC3AFDE08A789
S123C5200008DF089B0A970A7A000B860C970D7EC67FDE08A70008DF089B0A970A7A000BFD
S123C540860E970D7EC67F9B0A970A7A000B8614970D7EC67FDE08A70008DF089B0A970A4E
S123C5607A000B8610970D7EC67FDE08A70008DF089B0A970A7A000B8612970D7EC67F816E
S123C58007270B81082707810A27037EC3AFDE08A70008DF0897077A000B9B0A970A860D8A
S123C5A0B7000D7EC67F8130252D81392229DE08A70008DF089B0A970A7A000B7A000727F9
S123C5C0037EC67F7D000B26078616970D7EC67F860B970D7EC67F7EC3AF810127037EC304
S123C5E0AFDE08A70008DF089B0A970A7A000B860F970D7EC67F814F2707815027037EC30B
S123C600AFDE08A70008DF089B0A970A7A000B26078616970D7EC67F860B970D7EC67F8177
S123C6200127037EC3AF9B0A970A7A000B8615970D7EC67F814C2707815227037EC3AF9B8B
S123C6400A970A7A000B26078616970D7EC67F860B970D7EC67F9B0A27037EC3AF860097A2
S123C6600D7D000C2604C601D70296044C97049705CE000FC6153A4A26FCDF087EC67F7DB4
S123C680000C27037EC7017D000126037EC7017D0002266DB6100A84042609960581012354
S123C6A0604A2010B6100A8402261796054C91042302204D9705860197027F00007F000140
S123C6C0203F7D0003273AB6100A841026070F7F00037EC1A7B6100A842026088601970C42
S123C6E097022013B6100A840826167D000427119605BDCA36860197027F00017F0003207F
S123C700007D000C26447D0002273F7D000426298601BDCDA9B74000860CBDCDA9B7400000
S123C720CEC144BDCD9886C0BDCDA9B74000CEC155BDCD987F000220117F0002860CBDCD3B
S123C740A9B74000BDCB5BBDCA74960C810126697D000226647D0001275FB6100A8402261B
S123C7600996064C81112312204FB6100A8404261796064A81012402203F9706860197024F
S123C7807F00017F000020317D00032717B6100A8420261086FF970C860197027F00017F96
S123C7A000032015B6100A8418260E8602970C860197027F00017F0003960C8101263F7D4A
S123C7C00002273A8601BDCDA9B74000CEC166BDCD989606BDCD6EBDCD45BDCD8F17BDCD0D
S123C7E08F86C0BDCDA9B74000CEB61AC61B96064A27033A20FABDCD987F00022000960CEE
S123C80081FF27037EC8A37D000227037EC8A37D000126037EC8A3B6100A84022606B640E7
S123C820014C200BB6100A84042644B640014AC610BDCDA9F74000F64000C440260E81301A
S123C84024028639813923108630200C81202402867F817F23028620BDCDA9B74001C61088
S123C860BDCDA9F740007F0001863297002034B6100A84082605BDC9FF20EB7D0003272346
S123C880B6100A84102607BDCC1F86012008B6100A8420260E4F970C4C97027F00017F002E
S123C8A0032000960C81FF2658960227547F00028601BDCDA9B740008623BDCD8F9606BD51
S123C8C0CD6EBDCD45BDCD8F17BDCD8F8620BDCD8F8620BDCD8FCEB610C61B96064A2703FE
S123C8E03A20FABDCAF786C0BDCDA9B74000BDCD988685BDCDA9B74000860EBDCDA9B740DD
S123C90000960C810226709602276C7F00028601BDCDA9B74000D60E4F8F960EBDCD45BD09
S123C920CD8F17BDCD8F863ABDCD8FC604378620BDCD8FA60008BDCD45BDCD8F17BDCD8F08
S123C940335A26E986C0BDCDA9B740003C3332BDCD45BDCD8F17BDCD8F863ABDCD8FC6046B
S123C960378620BDCD8FA60008BDCD45BDCD8F17BDCD8F335A26E9960C8102264A7D000247
S123C98026457D00012740B6100A84022606960E8B08200BB6100A84042612960E8008970C
S123C9A00E860197027F00017F0000201A7D00032715B6100A8420260E8600970C86019761
S123C9C0027F00017F0003B6100A843E813E260C96038105220B8B019703200A7F0003208E
S123C9E0058601B700013E7EC2DD8640B7102596008B01816426054FC601D70197003B866A
S123CA0014BDCDA9B74000BDCDA9B64000847F810826098614BDCDA9B74000398110260933
S123CA2086C0BDCDA9B7400039815026088685BDCDA9B7400039B1000426107A00047A00F9
S123CA4005FC0008830015FD000839C615CE000F4A27033A20FAF60004F0000586153DA606
S123CA6015A700085A26F87A0004FC0008830015FD000839A600810227248104270139C6FE
S123CA80C0BDCDA9F740000808A600CECB39814F2708CECB4A8150270139BDCD9839083C2D
S123CAA01838E60008C0073ABDCC898C0000270C86C0BDCDA9B74000BDCD9839183C388685
S123CAC0C4E600C107270E8001C10827088001C10A27028001BDCDA9B74000E60008C10A59
S123CAE02715C10722022026A60008BDCD8F862DBDCD8FC1082317A60008BDCD8FA60008B9
S123CB00BDCD8FA60008BDCD8F862DBDCD8FA60008BDCD8FA60008BDCD8FA60008BDCD8F10
S123CB20A60008BDCD8FA60008BDCD8FA60008BDCD8FA60008BDCD8F392A204F7574206F8B
S123CB40662052616E6765202A00204E756D01726F205072697601212020008601BDCDA905
S123CB60B740008623BDCD8FB600058B30813A26028600BDCD8F8620BDCD8FCE000FB600AE
S123CB8005C6154A27033A20FA0808A60008BDCD8FA600090909BDCD8F862FBDCD8FA600C4
S123CBA008BDCD8FA600080808BDCD8F8620BDCD8FE60058585858A60180301B8112242C1F
S123CBC0A6000881302703BDCD8FA60008BDCD8F863ABDCD8FA60008BDCD8FA60008BDCD10
S123CBE08F8661BDCD8F866DBDCD8F39811227038B8819BDCD4581302703BDCD8F17BDCD10
S123CC008F0808863ABDCD8FA60008BDCD8FA60008BDCD8F8670BDCD8F866DBDCD8F390FA7
S123CC208685BDCDA9B74000CEB610C61B96064A27033A20FAC603BDCDA9B64001A1002727
S123CC4006BDCD18BDCD2D085A26EC8689BDCDA9B74000C607BDCDA9B64001A1002706BD42
S123CC60CD18BDCD2D085A26EC86C0BDCDA9B74000C610BDCDA9B64001A1002706BDCD18C0
S123CC80BDCD2D085A26EC0E39183C3736F6B61018CEB6105D272F373C183CC60AA60018ED
S123CCA0A100260F0818085A26F338C60A3A18383320161838C61B183A38335A26D9323358
S123CCC01838BDCCCE39CE00003233183839183C3736F6CE9918CECE995D2727373C183CD7
S123CCE0C60AA60018A100260F0818085A26F338C60A3A183833200E1838C61B183A383350
S123CD005A26D9CE00003233183839183C18CE06DA180926FC183839368616B7103BA70099
S123CD204CB7103BBDCD0B4FB7103B3239368602B7103B3236A7008603B7103BBDCD0B4F12
S123CD40B7103B32393C36CECD5E16545454543AE60017CECD5E33C40F3AE6003839303169
S123CD603233343536373839414243444546373C16CECD7A3AA6003833390001020304053D
S123CD800607080910111213141516171819207D40002BFBB7400139A600084D2601397D98
S123CDA040002BFBB7400120EF7D40002BFB39CEC00018CEC19E18FF000818CECE19CC005B
S123CDC000FD00058601B70007A600B4000727028601F60006C47F183C183A18E6001838C4
S123CDE0F70004B80004F60005595959F70004B8000444790006790005740007250986014A
S123CE00B10007270920C28680B7000720BBBC000827030820B3DC053900000101000001BF
S123CE200101010000010100000000010100000101010100000101000001010000010100DD
S123CE400000000101000001010101000001010000000001010000010100000101000001BF
S123CE6001010100000101000000000101000001010101000001010000010100000101009D
S123CE80000000010100000101010100000101000000000101000001013036353733383213
S117CEA03031374D61747420202020202020202020202000CC
S123FFD6C1A7C1A7C1A7C1A7C1A7C1A7C1A7C1A7C1A7C1A7C1A7C1A7C1A7C9EAC1A7C1A73C
S10DFFF6C1A7C1A7C1A7C1A7C1A7F5
S9030000FC
